:100000000C9499030C94D1030C94D1030C94D10358
:100010000C94D1030C94D1030C94D1030C94D10310
:100020000C94D1030C94D1030C94E30E0C94250E84
:100030000C9439190C94D1030C94D1030C94D10372
:100040000C94D1030C94D1030C94D1030C94D103E0
:100050000C94D1030C94FB180C94D1030C94D10391
:100060000C94D1030C94D1030C94D1030C94D103C0
:100070000C94D1030C94D1030C94D1030C94D103B0
:100080000C94D1030C94D1030C94D1030C94D103A0
:100090000C94D1030C94D1030C94D1030C94D10390
:1000A0000C94D1030C94D1030C94D103CC064007DB
:1000B000D4069E06A206D806A506DB06E606B0060E
:1000C0003607B406EA06B806EE061807BC06F206BE
:1000D0002207C206F8060207A906DF06AC06E206FA
:1000E000C706FD060E072E0730079A06D0064907F9
:1000F0006F077507630769077B07810787077E0816
:100100007E08B008B0082F09470A470A470A4B097A
:10011000BF09D009D009350C5C0C0D0E5C0C0D0E1E
:10012000A80CCB0C0D0EC10DD10D3A123D12791257
:1001300092129912A412A712A712A7127313731383
:10014000DB12DE12E212071329132C132F135313A1
:10015000AE1BA41BBB1B091C0F1C0F1C091C0F1C76
:100160000F1CDC1B0F1CE61BF01B0F1C0F1C0F1CB5
:100170000F1C091C0F1C0F1C091C0F1CC91B0F1C7A
:100180000F1C0B1C0B1C0B1C0B1C0B1C0B1C0B1C33
:100190000B1C0B1C0D1C0F1CAE1BA11B0F1C0F1CE2
:1001A0000F1C0F1C0F1C0F1C0F1C0F1C0F1C0F1CF7
:1001B0000D1C0F1C0F1C091C0F1CFE1BFE1BFE1B25
:1001C000FE1BFE1BFE1BFE1BFE1BFE1B0D1C000070
:1001D000000000000000000000000000000000001F
:1001E000000000000000000000000000000000000F
:1001F00000007E0F00D4FFFFFFC700000078000062
:100200000000000000002A2B280000000000000071
:1002100000000000000000000029000000002C1E6B
:100220003420212224342627252E362D3738271E28
:100230001F202122232425263333362E37381F044E
:1002400005060708090A0B0C0D0E0F1011121314E6
:1002500015161718191A1B1C1D2F3130232D3504A4
:1002600005060708090A0B0C0D0E0F1011121314C6
:1002700015161718191A1B1C1D2F3130354C050186
:100280000980A101850319012AB700150126B700CD
:10029000950175108100C0050C0901A101850419A3
:1002A000012AA002150126A002950175108100C047
:1002B00005010906A1018506050719E029E71500D2
:1002C00025019508750181020507190029EF150020
:1002D000250195F07501810205081901290595058B
:1002E00075019102950175039101C00660FF0961D6
:1002F000A1010962150026FF0095207508810209F9
:1003000063150026FF00952075089102C0050109BC
:1003100006A101050719E029E715002501950875D3
:100320000181029501750881010507190029FF1552
:100330000026FF00950675088100050819012905AA
:10034000150025019505750191029501750391012F
:10035000C009025B00030100A0FA090400000103C8
:100360000101000921110100012244000705810358
:100370000800010904010002030000000921110125
:100380000001222200070582032000010705030364
:1003900020000109040200010300000009211101ED
:1003A0000001226D000705840320000112010002F4
:1003B0000000000800F178AD020001020001120304
:1003C0004100640065006C0068006500690064001D
:1003D0000000120366006C006F006F006F006B007E
:1003E0006100790000000403090429003A003B0081
:1003F0003C003D003E003F00400041004200430001
:100400004400450068004B000000000000000000B0
:1004100000000000000000000000000000000000DC
:1004200000000000000035001E001F002000210019
:100430002200230024002500260027002D002E0086
:1004400031004C002B0014001A00080015001700A2
:100450001C0018000C00120013002F0030002A00AE
:100460004A00E00004001600070009000A000B0023
:100470000D000E000F0033003400280000004D0076
:10048000E1001D001B00060019000500110010000E
:10049000360037003800E500000052004E00E00052
:1004A0000000E20000002C00215200002C0000009F
:1004B000E60000000000500051004F00A600680058
:1004C00069006A006B006C006D006E006F007000C8
:1004D0007100720073004600A900000000000000D7
:1004E000000000000000000000000000000000000C
:1004F000000000000000000001003A003B003C004A
:100500003D003E003F0040004100420043004400E7
:100510004500010049000100010001000100010047
:1005200001004A004E004B004D0001000100010097
:100530004C000578E300010001000100010001000A
:100540005000510052004F0001000100AE000000B9
:10055000A8000100010001000100010001000100EC
:10056000010001000100010001000000AE00AA002E
:100570000100000001000000010001000000010076
:100580000000010000000000AC00AD00AB00010065
:100590000100010001000100010001000100010053
:1005A0000100010001000100010001000000000045
:1005B000000000000000000000000000000000003B
:1005C0000000000000000000000001000100010028
:1005D0000100010001000100010001000100010013
:1005E0000100010001000100010001000100010003
:1005F00001000100010001000100010001000100F3
:1006000001000100010001000100010001000100E2
:1006100001000100010001000100010001000100D2
:1006200000000100010001000100010001000100C3
:1006300001000100010001000100010000000100B3
:1006400001000100000001000000010001000000A5
:100650000100000001000000000001000100010095
:100660000100010001000100010001000100010082
:100670000100010001000100010001000100000073
:10068000000000000000000000000000000000006A
:100690000000000000000000000000000100010058
:1006A0000100010001000100010001000100010042
:1006B0000100010001000100010001000100010032
:1006C0000100010001000100010001000100010022
:1006D0000100010001000100010001000100010012
:1006E0000100010001000100010001000100010002
:1006F00001000000010001000100010001000100F3
:1007000001000100010001000100010001000000E2
:1007100001000100010000000100000001000100D3
:1007200000000100000001000000000001000100C5
:10073000010011241FBECFEFDAE0DEBFCDBF04B64B
:1007400003FE18C08091890290918A02A0918B02C9
:10075000B0918C028730904BA740B04B59F4109267
:10076000890210928A0210928B0210928C02E0E0B1
:10077000F8E3099511E0A0E0B1E0E0E3F3E402C0A2
:1007800005900D92AC36B107D9F722E0ACE6B1E0A6
:1007900001C01D92A938B207E1F70E9462100C94C3
:1007A00096210C940000A6E0B0E0E9EDF3E00C9493
:1007B000612149835A8349815A81992361F0222317
:1007C00051F0CA010E944B14182F682F89819A8119
:1007D0000E94651604C0CA010E943116182F698153
:1007E0007A81812F0E947E1E2696E3E00C947D2163
:1007F000ABE1B0E0EEEFF3E00C9460214E8B5F8B49
:10080000688F798F8A8F9B8F192F911110921F02F9
:10081000DE011F9687E0FD0111928A95E9F786E0D7
:10082000FE01769601900D928A95E1F70A8D0023DC
:1008300041F021E04F85588969897A89C8010E9471
:10084000D3030B8B1C8B87E0FE013F96DE011896CD
:1008500001900D928A95E1F7CE0108960E94AA14A4
:1008600081112CC087E0FE013896DE0111960190BF
:100870000D928A95E1F76C85662301F12091E301E1
:1008800030E0C90101968770992740911C0250E021
:100890008417950761F16D8397E0929FD001939F34
:1008A000B00D1124AC51BE4FFE01319601900D9256
:1008B0009A95E1F78093E3010E94E81317E0809195
:1008C0001C029091E3018917F9F0189FC0011124CF
:1008D0008C519E4F0E94AA148823B1F080911C0273
:1008E00090E001968770992780931C02E8CF0E94C0
:1008F00009171092E30110921C02ECEDF1E087E081
:10090000DF011D928A95E9F76B96E4E00C947C2157
:100910000E9409172FEF84E39CE021508040904013
:10092000E1F700C000009CE088E10FB6F894A895BC
:10093000809360000FBE90936000FFCFA8E0B0E00E
:10094000E4EAF4E00C945221FC018481882309F448
:10095000DFC57F0121E040815181628173819581F2
:100960000E94D3038C01F7018581882309F4BAC161
:10097000980137572038310508F032C1003108F0AE
:10098000E2C28FEF93E00E9493208111DCC230E736
:10099000A32E33E0B32E002379F0A114F4E0BF06B8
:1009A00009F4D1C2C5010E949320811101C00150F8
:1009B0002FEFA21AB20AEFCFCE0101962C0188E0E8
:1009C000F20111928A95E9F72AE0322E85010F5F34
:1009D0001F4FC5010E94932089831A82882309F43E
:1009E000B2C2813009F041C06501F2E0CF0ED11CE6
:1009F000C8010E9493208A83882309F4A4C29FEF30
:100A0000980F933060F423E0A20EB11CC6010E943F
:100A100093208B83882309F496C21C8229C08430DA
:100A200031F54E0133E0830E911C02E010E05601D7
:100A30008FEFA81AB80AC6010E949320F40181938F
:100A40004F01882309F47FC28C3741F4E2E0F0E0E3
:100A5000EC0FFD1FE00FF11F10820AC00F5F1F4F48
:100A600065010730110519F76EC2580101C0560122
:100A70008201F8012081222309F4A8CF213009F056
:100A800053C08181813081F46801F2E0CF0ED11C26
:100A9000F8018281893319F460E570E002C060E0FA
:100AA00070E00E946A1815C0823049F46801F2E0D3
:100AB000CF0ED11CF80182810E948D170AC08330AD
:100AC00051F46801F2E0CF0ED11CF80182810E943E
:100AD0003C17860182C0843019F00F5F1F4F7DC024
:100AE000F80122810E5F1F4F80E090E030E020533C
:100AF00031092A30310568F4389EA001399E500D25
:100B00001124C901840F951F0F5F1F4FF801208129
:100B1000EDCF009709F461C0EFE9FFE03197F1F7FD
:100B200000C000000197F5CFE22FF0E0E250FE4F49
:100B30002490822F86958695869590E0FC01E2515F
:100B4000FE4F64902770712C022E02C0759467943A
:100B50000A94E2F7F1E06F227724FC01E252FE4FA3
:100B60008490912C022E02C0959487940A94E2F707
:100B700031E083229924FC01E253FE4FC490D12C32
:100B800002C0D594C7942A95E2F781E0C822DD24FB
:100B90006114710419F081EE0E948D178114910483
:100BA00019F086EE0E948D1760E070E0822D0E94A1
:100BB0006A188114910419F086EE0E943C176114A2
:100BC000710419F081EE0E943C17C114D10429F080
:100BD00060E070E08CE20E946A180F5F1F4F49CFFF
:100BE000023098E7190709F470C058F40115F8E7C6
:100BF0001F0791F0013028E7120709F073C080E069
:100C00000CC0043038E7130709F446C068F005301B
:100C1000E8E71E07C9F066C083E00E9423108091B8
:100C2000B1010E94B31C8FC18091B101982F96959C
:100C30009695969549F1915E990F990F990F877046
:100C4000892B8093B10114C09091B101892F8695B1
:100C5000869586958F5F8F719770843008F03FC0BE
:100C6000880F880F880F892B8093B1018091B10183
:100C7000887F91E009F490E08091B10190FB80F9C8
:100C80008093B1010E94B31C8091B1018695869535
:100C900086950E94111C57C12091B101822F869523
:100CA00086958695482F50E04330510554F48F5F68
:100CB000982F990F990F990F822F8770892B809306
:100CC000B1018091B1018160DBCF8091B10180FFE2
:100CD00003C00E943D1037C10E944A1034C1909356
:100CE000B101C4CFF801E851FC47E730F10508F441
:100CF000E6C0882309F43BC110924C02980130579A
:100D00002332310508F00CC184E090E00E949B2062
:100D10009093540280935302F801E150F047E2327D
:100D2000F10520F4EA5AFF4F0C942B2180915302D5
:100D30008160ACC0809154028860B4C0809153023D
:100D40008260A4C08091530220C0809153028860C9
:100D50009DC0809154021EC0809154028260A2C046
:100D600080915302806192C08091530280628EC054
:100D70008091530280648AC00E94091780915302B7
:100D8000806884C080915302886084607FC08091B5
:100D900054028260816086C0809153028E7F76C04B
:100DA00080915402877F7EC0809153028D7F6EC0F8
:100DB0008091530220C080915302877F67C0809149
:100DC00054021EC0809154028D7F6CC080915302EA
:100DD0008F7E5CC0809153028F7D58C080915302FA
:100DE0008F7B54C00E940917809153028F774EC0A9
:100DF00080915302877F8B7F49C0809154028D7F01
:100E00008E7F50C08091530282FB222720F991E00F
:100E1000922790FB82F990FB83F938C080915402AD
:100E2000982F909591708E7F892B90FB81F93AC015
:100E30008091530286FB222720F991E0922790FBB4
:100E400086F924C00E9409178091530287FB22274C
:100E500020F991E0922790FB87F918C061E001C06A
:100E600060E08EE090E00E94B1201EC080915302AD
:100E700084FB222720F991E0922790FB84F906C099
:100E800080915302982F909590FB80F980935302A4
:100E90000BC08091540283FB222720F991E0922716
:100EA00090FB83F980935402609153027091540235
:100EB00084E090E00E94CF200E94091744C0E858C7
:100EC000FF4F0C942B2106E221EE41EE6AE17CE714
:100ED00023C007E225EE45EE6BE17CE71DC006E28C
:100EE00021EE40EE68E17CE717C007E225EE44EE14
:100EF00069E17CE711C006E221EE42EE6CE17CE79D
:100F00000BC007E225EE46EE6DE17CE705C008E286
:100F100021E045EE6EE17CE7C7010E945B1A13C039
:100F20000631FCE71F0791F5809182028A7A91E0F1
:100F300009F490E090936E01811117C089E20E943C
:100F400090190E94412080911D02877009F4E0C22F
:100F5000F7018581882309F4DBC28091540282FF66
:100F6000D7C282E00E94CC16D3C285E3E8CF063117
:100F70002CE7120709F0B3C280916E01811104C001
:100F800089E20E946219DDCF85E3FBCF07373CE79A
:100F9000130711F481E0B1C208379CE7190709F47F
:100FA000ABC29801205E324520323105A8F4811190
:100FB00015C00F7181E090E09C0102C0220F331F29
:100FC0000A95E2F78901622F83E090E00E94B12048
:100FD000802F0E940617B7CF8823D9F103303CE752
:100FE000130721F140F401159CE7190789F001303E
:100FF0001C4711F12EC00B35FCE71F0739F10C35EA
:101000002CE71207D9F00A351C4719F581E01FC0FB
:101010000E9409178FEF94E3ECE081509040E0408C
:10102000E1F700C000000E94D7188DCF6FEF7FEF6F
:1010300080E090E00E94CF200E94880480915402BA
:1010400082FB882780F991E0892701C080E00E9417
:10105000E316F701858100811181882349F0C801D9
:101060000E944B14D82E682FC8010E94651604C038
:10107000C8010E943116D82EB8018D2D0E947E1E07
:101080000E948C1E8C01A82EF701B5809680929448
:101090009FE0992280911D02877001F1BB20F1F041
:1010A000812F807F803469F080E2800F8830B0F03B
:1010B000812F807E803229F4F1E0F01778F49920B6
:1010C00069F08091540282FF09C082E00E94CC1630
:1010D00080911D028770DD24D3948111D12CC12E03
:1010E000C2948FE0C8228C2D90E08C30910508F0DE
:1010F000CEC1FC01E158FF4F0C942B21812F807F42
:101100001F70882311F01295107FBB20B9F01123B6
:1011100009F4ABC180E2800F883010F0A11006C046
:1011200090918202192B1093820205C090911F02A8
:10113000192B10931F020E94412097C1802F0E94FB
:101140003C17112309F4A3C1005E083080F1AA20E6
:1011500071F1109590911F02192310931F022AC05C
:10116000812F807F1F70803211F01295107FAA208E
:1011700029F021E0A21609F44DC058C08091540214
:1011800082FD1BC0BB2069F0112339F0309182022F
:10119000312B309382020E94412080E00E948D1703
:1011A00076C180E00E943C17112309F470C1812FA1
:1011B0000E943A200E9441206AC1BB2081F0992000
:1011C000C9F131E0931263C130911E02812F832354
:1011D000181709F45CC1312B30931E0258C19110CD
:1011E00056C1812F0E942B1730911E02812F83231D
:1011F00029F0812F8095382330931E0220916F01B2
:10120000812F822309F443C1312F3095232320936A
:101210006F013DC1BB2029F085E0891508F437C175
:1012200009C094E0991508F432C115C0BB2031F013
:1012300091101BC1812F0E94321729C1992059F0AA
:10124000093309F021C1EFEFF7EE23E0E150F04060
:101250002040E1F717C1812F0E942B1718C1812F61
:1012600086958695837019F0813059F010C1BB20A6
:1012700019F0C801937002C080E090E00E94EC1960
:101280000CC1BB2019F0C801937002C080E090E04F
:101290000E94C71902C1812F8370A9F5B110FBC04C
:1012A000402F429546954770440F440F802F8F7012
:1012B00090E09C01042E01C0220F0A94EAF704FF7B
:1012C00008C08FE090E001C0880F4A95EAF780954A
:1012D00001C080E0169516951370123069F088F4FD
:1012E00090918302113019F0822B892302C0922B36
:1012F000892B0E940617CFC0822B909183028927E9
:10130000F8CF822BF6CFBB2019F0812F817001C05E
:101310008695882309F4BFC0402F429546954770B3
:10132000440F440F802F8F7090E09C01042E01C069
:10133000220F0A94EAF704FF08C08FE090E001C092
:10134000880F4A95EAF7809501C080E016951695BA
:101350001370123059F078F490919301113019F014
:10136000822B892309C0922B892B06C0822B909156
:101370009301892701C0822B0E949A168CC01F708E
:10138000BB2039F0812F0E94FA16802F0E9432175D
:1013900082C0802F0E942B17812F0E94BF167BC016
:1013A000802F32EFA31681F13A1538F090EFA9168D
:1013B00059F0E1EFAE1619F154C0F3EFAF1659F141
:1013C00024EFA216C1F04DC0BB2081F034E03915E6
:1013D00008F45DC01F7181E090E0012E01C0880F0C
:1013E0000A94EAF790919301892720C085E0891536
:1013F00008F44DC0EFCF8091540282FD1AC0BB208B
:1014000029F0812F8F7120C0BB20D9F3812F8F71DC
:101410000E94BF163CC0BB2041F01F7181E0012E2D
:1014200001C0880F0A94EAF701C080E00E949A1672
:101430002EC0BB2061F0812F8F7198E0899F9001B1
:101440001124236020931D020E94FA1620C081E01F
:101450000E94CC16E1E0E915D0F482E00E94CC169F
:1014600016C0BB2021F0992061F2802F97CE9920E1
:1014700069F2893349F4FFEF27EE33E0F150204061
:101480003040E1F700C00000802F0E943C1788EF39
:101490008C0D843010F40E94111ADD20A9F0809187
:1014A0001D0280FD11C0F7011582869586958695EF
:1014B0000E94FA16C7010E949E0480911D02869523
:1014C000869586950E94BF1620E0F70140815181E4
:1014D00062817381848195810E94D30319C007378B
:1014E000ECE71E0711F481E00BC00837FCE71F078B
:1014F00009F057CD82E004C082E00E94FA1602C0D3
:101500000E94BF1643E062E081E00E949D161BCD61
:101510002896E2E10C946E2180917D0187FF11C035
:101520008091E80082FD05C080917B018111F8CF98
:1015300011C08091E8008B770BC080917B018823DC
:1015400049F08091E80080FFF8CF8091E8008E7725
:101550008093E8000895982F973068F59093E900FC
:10156000981739F07091EC002091ED005091F00047
:1015700003C0242F762F50E021FD02C09F5FECCFE7
:101580003091EB003E7F3093EB003091ED003D7FDA
:101590003093ED003091EB0031603093EB007093AD
:1015A000EC002093ED005093F0002091EE0027FD19
:1015B000E5CF80E008958F708093E90081E0089581
:1015C00020918301309184012617370748F0611577
:1015D000710539F42091E8002E772093E80001C0CE
:1015E000B901FC0120E06115710579F180917B0161
:1015F0008823F1F18530F1F18091E80083FD3CC052
:101600008091E80082FD2EC08091E80080FFEBCF42
:101610002091F3008091F20090E0922B611571050A
:1016200051F08830910538F421912093F1006150F8
:1016300071090196F3CF21E0089709F020E080912D
:10164000E8008E778093E800CECF2111CFCF0AC07B
:1016500080917B01882361F0853061F08091E80002
:1016600083FD0AC08091E80082FFF2CF80E00895F8
:1016700082E0089583E0089581E00895089543E0AD
:1016800050E0BC0184E00E948518089540E250E0DB
:10169000BC0184E00E9485180895AAE2B0E0E3E569
:1016A000FBE00C946121EDE7F1E085E891E0209109
:1016B000F10021938E179F07D1F780917E0183302F
:1016C00009F463C030F4813071F0823009F4A2C0B3
:1016D000B9C08A3009F48EC08B3009F46EC08930ED
:1016E00009F0B0C020C080917D01813A09F0AAC004
:1016F0008091E800877F8093E8008091810190913C
:101700008201892B21F468E081E791E003C060E069
:1017100080E090E070E00E94E00A8091E8008B7722
:101720008093E8008FC080917D01813209F08AC0EA
:101730008091810190918201009719F0029709F040
:1017400081C08091E800877F8093E8008091E80065
:1017500082FD05C080917B018111F8CF73C020917B
:10176000F3008091F20090E0922B029731F4809187
:10177000F100813011F0863021F48091F1008093E6
:1017800001018091E8008B7759C080917D01813AF9
:1017900009F058C08091810190918201892B09F054
:1017A00051C08091E800877F8093E8008091E80035
:1017B00080FFFCCF809102013CC080917D0181328D
:1017C00009F040C08091810190918201892BD1F56F
:1017D0008091E800877F8093E8000E948C0A81E076
:1017E00090917F01911101C080E0809302010E94DD
:1017F000091728C080917D01813221F58091E80090
:10180000877F8093E8000E948C0A809180018093FA
:10181000000118C080917D01813AA1F48091E80017
:10182000877F8093E8008091E80080FFFCCF809163
:1018300000018093F1008091E8008E778093E800AA
:101840000E948C0A8091E80083FFE7C180917D01AE
:1018500090917E01492F50E04A30510508F0DDC1DA
:10186000FA01E557FF4F0C942B21803821F0823884
:1018700009F0D3C108C08091790190917A01992330
:1018800089F082600FC0809181018F70873008F0ED
:10189000C4C18093E9008091EB0085FB882780F923
:1018A0001092E9009091E800977F9093E800809370
:1018B000F1001092F10071C1282F2D7F09F0ADC108
:1018C000882319F0823061F0A8C180917F018130B6
:1018D00009F0A3C1933009F080E080937A012EC013
:1018E00080917F0181112AC0809181018F702FEF3B
:1018F000280F263008F091C18093E9002091EB0079
:1019000020FF1CC0933021F48091EB00806214C052
:101910009091EB0090619093EB0021E030E0A90101
:1019200002C0440F551F8A95E2F74093EA001092D7
:10193000EA008091EB0088608093EB001092E90050
:101940008091E800877F8093E8000E948C0A65C13F
:10195000811163C110917F011F778091E30080782E
:10196000812B8093E3008091E800877F8093E800DB
:101970000E948C0A8091E80080FFFCCF8091E300F8
:1019800080688093E300111102C082E001C083E00F
:1019900080937B0142C18058823008F03EC1209183
:1019A0007F01309180012C3D53E0350779F583E0CC
:1019B0008A838AE289834FB7F894DE01139620E088
:1019C0003EE051E2E32FF0E050935700E49120FF16
:1019D00003C0E295EF703F5FEF708E2F90E0EA302A
:1019E00010F0C79601C0C0968D939D932F5F243150
:1019F00049F74FBF8091E800877F8093E8006AE253
:101A000070E0CE0101960E94E00AB5C0809181018C
:101A100090918201432F552743305105A9F068F476
:101A20004130510509F408C14230510509F0F5C0B3
:101A30008BE590E0E1E5F3E04BC04132510529F13F
:101A40004232510589F1E9C0C901992781309105D8
:101A5000A1F058F0029709F0E0C0EEEBF3E0E4915A
:101A60008E2F90E0EEEBF3E030C0E6EEF3E0E49191
:101A70008E2F90E0E6EEF3E028C0E2EDF3E0E49193
:101A80008E2F90E0E2EDF3E020C08330910508F066
:101A9000C4C0880F991FFC01E95EFE4F0190F081E0
:101AA000E02D89E090E014C08330910508F0B5C0C6
:101AB000FC01EE0FFF1FEF5EFE4F0190F081E02D65
:101AC000DC01A25FBE4F8C9190E0009709F4A5C0A5
:101AD0002091E800277F2093E80020918301309136
:101AE00084018217930708F49C0140E02115310519
:101AF00089F180917B01882309F43DC08530D9F1BB
:101B00008091E80083FD37C08091E80082FD2FC0FE
:101B10008091E80080FFEACF4091F3008091F200CD
:101B200090E0942B2115310559F08830910540F44F
:101B300044914093F1003196215031090196F2CF42
:101B400041E0089709F040E08091E8008E778093AB
:101B5000E800CCCF4111CDCF0AC080917B01882312
:101B600051F0853041F08091E80083FD04C0809100
:101B7000E80082FFF2CF8091E8008B778093E80045
:101B80004CC0803809F049C08091E800877F80937D
:101B9000E80080917C018093F1008091E8008E77CD
:101BA000D2CE81113AC080917F0190918001992716
:101BB00002979CF58091E800877F8093E800109160
:101BC0007F0110937C010E948C0A111106C0809144
:101BD000E30087FD02C081E001C084E080937B01C7
:101BE00042E061EC81E00E94AB0A42E261EC84E0F9
:101BF0000E94AB0A42E261EC82E00E94AB0A42E240
:101C000060EC83E00E94AB0A80917B01843011F08C
:101C100081E001C082E0809303018091E80083FFAE
:101C200010C08091E800877F8093E8008091EB00EE
:101C300080628093EB0005C082E190E0ECEAF3E083
:101C400047CFAA96E3E00C947D211F920F920FB626
:101C50000F9211242F933F934F935F936F937F9332
:101C60008F939F93AF93BF93CF93DF93EF93FF93A4
:101C7000C091E900CF708091EC00D82FD17080FD29
:101C8000D0E81092E9008091F000877F8093F00007
:101C900078940E944D0B1092E9008091F0008860CA
:101CA0008093F000CD2BCF70C093E900FF91EF91AE
:101CB000DF91CF91BF91AF919F918F917F916F9164
:101CC0005F914F913F912F910F900FBE0F901F90FA
:101CD0001895E8EDF0E080818E7F80831092E2001D
:101CE0001092DA001092E100A0EEB0E08C918160D9
:101CF0008C9380818F77808319BCA7EDB0E08C91A5
:101D00008E7F8C9380818F7E8083109270010895E6
:101D1000A0E0B0E0EEE8FEE00C945C21C8EDD0E07D
:101D200088818F7E8883E7EDF0E080818160808309
:101D300084E082BF81E08093700188818E7F8883F8
:101D400002EE10E0F80110821092DA0081EEC82E47
:101D5000D12CF601108288818F77888388818068F2
:101D6000888388818F7D888319BC10927B011092B3
:101D70007C0110927A011092790190EEE92EF12CFB
:101D8000F70180818B7F808388818160888342E036
:101D900060E080E00E94AB0AF60180818E7F808344
:101DA000F801808181608083808188608083F70171
:101DB00080818E7F8083888180618883CDB7DEB704
:101DC000E8E00C9478211F920F920FB60F92112425
:101DD0002F933F934F935F936F937F938F939F9333
:101DE000AF93BF93EF93FF938091E10082FF09C00F
:101DF0008091E20082FF05C08091E1008B7F80939B
:101E0000E1008091DA0080FF2AC08091D80080FF35
:101E100026C08091DA008E7F8093DA008091D9000D
:101E200080FF18C080E189BD82E189BD09B400FE50
:101E3000FDCF81E080937B018091700181110FC003
:101E40000E94690E0E94880E8091E2008460809357
:101E5000E20005C019BC10927B01109270018091C4
:101E6000E10080FF1AC08091E20080FF16C08091DF
:101E7000E2008E7F8093E2008091E2008061809397
:101E8000E2008091D80080628093D80019BC85E080
:101E900080937B0183E0809303018091E10084FFC4
:101EA00037C08091E20084FF33C080E189BD82E1C8
:101EB00089BD09B400FEFDCF8091D8008F7D80934D
:101EC000D8008091E1008F7E8093E1008091E20054
:101ED0008F7E8093E2008091E20081608093E20037
:101EE00080917C01882311F084E007C08091E30099
:101EF00087FD02C081E001C083E080937B01809177
:101F00007B01843011F081E001C082E08093030105
:101F10008091E10083FF2CC08091E20083FF28C004
:101F20008091E100877F8093E10082E080937B01D4
:101F300010927C018091E1008E7F8093E10080917E
:101F4000E2008E7F8093E2008091E20080618093C6
:101F5000E20042E060E080E00E94AB0A8091F00085
:101F600088608093F00081E08093030180930201F8
:101F7000FF91EF91BF91AF919F918F917F916F9161
:101F80005F914F913F912F910F900FBE0F901F9037
:101F900018952091E4003091E50095E64091EC0021
:101FA000842F817040FF23C08091E80080FD1DC018
:101FB00080917B01882399F0853099F08091EB0026
:101FC00085FD11C04091E4005091E50024173507CC
:101FD00029F3915011F09A01E1CF84E0089582E055
:101FE000089583E0089581E0089580E00895409188
:101FF000E80042FFDDCF089586E090E00E94932044
:102000008093B10182FD05C08DE18093B1010E94F2
:10201000B31C8091B101282F26952695269530E096
:102020002430310524F0877088618093B10180915C
:10203000B10180FF04C086958695869501C080E039
:102040000E94111C0895843008F083E09091B10142
:102050009770282F220F220F220F922B9093B101FD
:10206000987F21E009F420E09091B10120FB90F9E4
:102070009093B1010E94111C08958091B10180FFDD
:1020800008C08E7F8093B1010E94B31C80E00E9443
:10209000111C08958091B10180FD13C0816080936F
:1020A000B101813019F489E08093B1018091B101CF
:1020B0000E94B31C8091B1018695869586950E94F9
:1020C000111C0895A6E2B0E0E8E6F0E10C9452217C
:1020D00085B7806885BF85B7806885BF84B7877FEF
:1020E00084BF0FB6F894A8958091600088618093B2
:1020F0006000109260000FBE90E080E80FB6F89488
:1021000080936100909361000FBE81E08093030192
:1021100089EB9CE190936D0180936C010E94690EA4
:102120000E94880E8091E20084608093E20078949F
:1021300080917B018823A1F01091E9001F7090919C
:10214000EC00892F817090FD80E8182B1092E90037
:102150008091E80083FD0E944D0B1F701093E900F1
:1021600082E084BD93E095BD9AEF97BD80936E00A9
:102170000E94421A811102C00E94571B0DE111E01A
:10218000D8018D918D018F3F11F00E94A61DB1E005
:1021900004321B07A9F704E211E0B3E3EB2EB1E030
:1021A000FB2EF80181918F018F3F11F00E94A61D37
:1021B000E016F106B1F78EE0E3EAF1E0DF01282F47
:1021C0001D922A95E9F7E5E8F1E0DF011D928A9575
:1021D000E9F780E090E00E949B20853E9E4F21F42D
:1021E0000E94421A811102C00E94CD1F82E090E03D
:1021F0000E9493208093490284E090E00E949B20FB
:1022000090935402809353020E94BD1DEFEFF6E7B6
:1022100021E0E150F0402040E1F700C000000E94C2
:10222000BD1D8091A30180FF08C06FEF7FEF80E0AC
:1022300090E00E94CF200E94D71883E090E00E9497
:1022400093200E9406173E9A469882E88093900059
:1022500089E1809391008FEF9FEF90939700809397
:1022600096000E94FC0F0E94FC0F84E091E0909386
:10227000500280934F028E010F5F1F4FA3E04A2E42
:10228000512C80917B01853009F044C080917B0105
:10229000853009F039C080917B01843039F180E0CC
:1022A0000E9423101092550288E190E0A0E40FB63E
:1022B000F894A895809360000FBEA093600083B748
:1022C000817F846083BF83B7816083BF7894889562
:1022D00083B78E7F83BF0FB6F894A8958091600076
:1022E000886180936000109260000FBE0E94BD1D47
:1022F000E3EAF1E081919191892B09F0FDC1B1E010
:10230000E13BFB07B9F7C2CF0E9409170E94FC0FFF
:102310000E94111A0E94BD1DE4E9EE2EE1E0FE2E9E
:10232000F3EA6F2EF1E07F2ED301F7012191319175
:102330008D919D918227932721E0E23AF20719F0CF
:10234000892BA1F305C0892B19F40E94A91F3FC056
:10235000312CD3018D909D903D01F701A080B1807B
:10236000A824B924A114B10449F1212CCC24C3948C
:10237000D12CC5018C219D21892BB9F029A23AA22B
:102380000E942D199CA38BA3F1E0FDA391E0940181
:102390002C213D21232B09F490E09EA349A15AA1B1
:1023A0006BA17CA18DA10E94F8032394CC0CDD1CB1
:1023B0002FE02212DECFD7018D929C923394B2E0AF
:1023C000EB0EF11CE7E03E12C4CF0E9421190E94DF
:1023D000111A9091A201891721F08093A2010E9405
:1023E000211980917B01843009F04BCF83E08093E9
:1023F000E9008091E80082FF44CF8091E80085FFEA
:1024000023C00E94C90F81111DC050E2C52ED12CDE
:10241000CE0101967C0109C08091F100D7018D9316
:102420007D01B1E0CB1AD10869F08091E80085FD0B
:10243000F3CF8091E8008B778093E8000E94C90F6A
:10244000882399F391E001C090E08091E8008B77B8
:102450008093E800992309F414CF2981822F90E01A
:10246000FC013197E331F10508F03DC1EB56FF4F18
:102470000C942B211A828CE0A3C08A81823009F44B
:1024800058C150F4813009F02EC10E9421199B835C
:102490008C837D836E8329C1833041F0843009F0C1
:1024A00022C11B821C821D821E821FC16B81DE0124
:1024B000119680E090E0262F30E0A901480F591FC7
:1024C0004730510508F011C1E62FE80FF0E0EE0F9C
:1024D000FF1FED55FE4F4081518113965C9313977A
:1024E00014964C931497019612968E30910529F705
:1024F000FCC08A81823019F0853051F0F4C06B81C4
:102500007C818D819E810E9431210E941E1AEDC026
:102510008091B10180FF03C00E943D10E6C00E947F
:102520004A10E3C04C816B818A810E94671B9D83A6
:1025300007C12D813E813227232732274C816B81B1
:102540008A810E94FB1AD1C00E94221BCEC08A81C0
:10255000813009F0C8C0283099F0293039F18B81D9
:10256000813009F0C2C08C81E3E08E9FC00111244C
:102570006FEF70E00E94F520862F0E942310B5C0F7
:102580008B81813029F0823009F0AFC01C82ADC050
:102590008091B101869586958695FFEF8F9FC0014A
:1025A0001124B2010E94F5206C839FC08091B1017B
:1025B0000E94B31C9AC020E12A8397C01A8280E946
:1025C0008B8393C0EA80FB80FE24EF24FE24AC8042
:1025D000B12C6801C70180599C4F9601201B310B1B
:1025E0002A153B0508F081C0A0E9EA16F10428F499
:1025F0000E949320F601848303C0D60114961C9296
:10260000BFEFEB1AFB0AEFEFCE1ADE0AE3CFEA8048
:10261000FB80FE24EF24FE24AC80B12C6801C701AE
:1026200080599C4F9601201B310B2A153B0508F061
:102630005CC0F0E9EF16F10428F4D60114966C9111
:102640000E94B120BFEFEB1AFB0AEFEFCE1ADE0AB1
:10265000E6CF0E94EB1A49C084E08A8346C0EA8034
:10266000FB80FE24EF24FE24AC80B12C6801C7015E
:1026700088969601201B310B2A153B05B0F5F8E42E
:10268000EF16F3E0FF0630F40E949320D601149673
:102690008C9302C0F6011482FFEFEF1AFF0A2FEFAE
:1026A000C21AD20AE4CFEA80FB80FE24EF24FE2483
:1026B000AC80B12C6801C70188969601201B310BB4
:1026C0002A153B0590F4A8E4EA16A3E0FA0620F4E4
:1026D000F60164810E94B120FFEFEF1AFF0A2FEF8D
:1026E000C21AD20AE8CF8FEF898340E250E0B801E6
:1026F00082E00E948518C5CD80917A01882309F473
:10270000C5CDE0E1E9BDF2E1F9BD09B400FEFDCFC0
:102710008091D8008F7D8093D8008091E000826006
:102720008093E0008091E00081FDFCCF0E940917BA
:10273000ADCD87E290E00E9493201B821C821D8217
:102740008E83D3CF20911C029091E30157E029178B
:10275000A9F030E0529FF001539FF00D1124EC518D
:10276000FE4F7181761306C07081781303C07581A6
:10277000741306C02F5F3F4F2770E9CF80E00895A4
:1027800081E008959091820280911F02892B90919F
:102790001E029923E1F0892B90910201913041F4BE
:1027A0009091530297FF04C09EE12AE232E003C0F9
:1027B00096E022E232E0F90120E0915028F03191D8
:1027C0003323D9F32F5FF9CF211110921E02089500
:1027D00080911C029091E301891719F08F5F877037
:1027E000FBCF0895CF93DF938091E20182958F70A4
:1027F00009F04EC08091E101882309F449C080911D
:102800001C024091E3015091DD016091DC01C09117
:10281000DE01D091DF0177E08417D1F190E0789F5D
:10282000F001799FF00D1124DF01AC51BE4F1496D9
:102830002C911497222349F111962C91119725136D
:1028400024C02C91261321C015962C911597211187
:102850001CC012962D913C9113972C1B3D0B283CCC
:10286000310598F48091E2018F7080618093E201DC
:10287000E651FE4F80818F70806180838CED91E006
:102880000E949E040E94E81303C001968770C4CF83
:10289000DF91CF910895CF92DF92FF920F931F9314
:1028A000CF93DF936C010091930180918302082BF9
:1028B000C3E0D0E010E0C8010C2E02C095958795CA
:1028C0000A94E2F780FD04C02197A8F7F12C09C013
:1028D000FC2EB6018C2F0E947E1E0E948C1E01973A
:1028E00099F38F2DDF91CF911F910F91FF90DF9082
:1028F000CF900895CF93DF93EC010E944B14BE015B
:102900000E947E1E0E948C1EDF91CF910895FC01D3
:1029100024812223D9F0808191810E947A1492959A
:102920009F70963079F010F4925001C09A50923016
:1029300068F4803F69F018F4883E40F409C0843F91
:1029400029F406C0883E20F0813F11F080E0089510
:1029500081E00895A4E1B0E0E0EBF4E10C945821AB
:102960008C0186E0F801DE011F9601900D928A9598
:10297000E1F7F8018481E5809CED892E91E0992EA4
:102980009091E001911120C0882309F463C1EE20E9
:1029900009F442C0C8010E948714F82E8823E1F18F
:1029A00087E0F801D40101900D928A95E1F78091BA
:1029B000E001813031F48091DC019091DD010E94D1
:1029C0007A140E94F21348C1F801D080C180A2801D
:1029D000B380F090E1012091DE013091DF01FF2012
:1029E00009F4E7C0A501421B530B483C510508F010
:1029F0009DC0882309F430C18091E201282F207FF7
:102A00009091DD01222361F09C1509F460C0C8019A
:102A10000E948714811163C0C8010E949E041AC1DC
:102A20009C1113C09091DC019D110FC0E1100DC0ED
:102A30008F7080618093E2018CED91E00E949E0492
:102A40008091E201F801868303C1E1103AC040E0C1
:102A50006C2D8D2D0E94A21340E06C2D8D2D0E94B7
:102A6000A213E82E8111F4C0DF86C88A8F85988969
:102A70000E947A14292F22952F70243020F49F7001
:102A8000223028F009C02A50223080F014C0992347
:102A900049F0811107C013C0992321F0F8019681F4
:102AA000907F69F0805E883030F409C0803F38F054
:102AB000815F833020F0C8010E949E04EF2CFE2C21
:102AC000CBC08091E20181608093E201C1C090910E
:102AD000DC019D119CCFE1109ACFF80198C0EE2047
:102AE00009F49ACF2091E201822F82958F7090E0B5
:102AF00002978CF08091DC019091DD0199878887A5
:102B0000BB86AA868091E0018C871D862E87CE0128
:102B100008960E949E0487E0F801ACEDB1E00190B8
:102B20000D928A95E1F70E94F21394C09091E20110
:102B3000292F207F51F48CED91E00E949E0487E0C4
:102B4000F40111928A95E9F783C0882309F484C0BF
:102B50008091DD018C110CC08091DC018D1108C0C9
:102B6000E11006C0F8019683C8010E949E046AC065
:102B7000C8010E948714882309F44ECFEE2009F47F
:102B80004BCF2091E201822F82958F7090E00297C7
:102B900014F28091DC019091DD019A838983BC82DB
:102BA000AB828091E0018D831E822F83CE0101963E
:102BB000B0CFA21AB30AF8ECAF16B10408F042C0C5
:102BC000882309F447C0FE2CEE2009F425CF80911C
:102BD000DD018C1129C08091DC018D1125C09091FF
:102BE000E20190FD18C0892F82958F70282F30E068
:102BF0002115310581F0F80196832F30310541F020
:102C00008F5F982F9295907F86818F70892B868316
:102C1000C8010E949E0487E0F801ACEDB1E001908C
:102C20000D928A95E1F718C0C8010E94871481119E
:102C300072CF8091E20181608093E201C8010E941D
:102C40009E040AC087E0F40111928A95E9F704C056
:102C5000F12C02C0FF24F3948F2D6496ECE00C94C9
:102C60007421292F973078F58F3068F590E03FE098
:102C7000239F800D911D1124682F677023E0969586
:102C800087952A95E1F7FC01EE0FFF1FE80FF91F6A
:102C9000EE54FE4F40E050E080E0219130E0062EFF
:102CA00002C0369527950A94E2F721703327042E47
:102CB00001C0220F0A94EAF7822B4F5F5F4F433027
:102CC000510559F7089580E00895292F973088F528
:102CD0008F3078F590E03FE0239F800D911D112407
:102CE000282F277051E001C0550F2A95EAF723E0FD
:102CF000969587952A95E1F7FC01EE0FFF1FE80FE7
:102D0000F91FEE54FE4F20E030E070E04081CB012F
:102D1000022E02C0969587950A94E2F781708195FC
:102D200084278523842781932F5F3F4F23303105EC
:102D300069F708958093930108959091930121E09C
:102D400030E0F90101C0EE0F8A95EAF7D90102C01F
:102D5000AA0FBB1F6A95E2F7BD016E2B01C0220FBF
:102D60004A95EAF7892F8623681303C0892F822B9F
:102D700003C02095822F89230E949A16089521E08E
:102D800030E001C0220F8A95EAF7209580919301E7
:102D900082230E949A16089590911D02809589239E
:102DA00080931D02282F277069F4981759F090918D
:102DB000540292FF07C08695869586950E94BF169D
:102DC00010921D0208959091540292FB222720F93F
:102DD000281779F080FB92F9909354026091530286
:102DE0007091540284E090E00E94CF2082E00E9423
:102DF000CC16089521E030E001C0220F8A95EAF751
:102E000080919301822B0E949A16089580938302E9
:102E100008951092820280910201813041F48091E4
:102E2000530287FF04C08EE1EAE2F2E003C086E0CD
:102E3000E2E2F2E0DF011D928A95E9F780E090E09E
:102E40000E94EC1980E090E00E94C71910921F02C6
:102E50000E9441200895882321F00E943A200E9478
:102E600041200895882339F090918202892B809324
:102E700082020E9441200895882309F44DC08238BF
:102E800059F40E94111A81FF47C089E30E949019EA
:102E90000E94412089E30CC0833879F40E94111A02
:102EA00080FF3AC083E50E9490190E94412083E58B
:102EB0000E9462190E9441200895843859F40E94AA
:102EC000111A82FF29C087E40E9490190E944120B4
:102ED00087E4EECF9CEF980F913A50F390E2980F71
:102EE000983050F4877091E001C0990F8A95EAF705
:102EF000892F0E943A20DECF9BE5980F933028F46B
:102F000080E090E00E94EC190895885A8B3120F4FB
:102F100080E090E00E94C7190895CF93882309F4B8
:102F2000D7C0C82F8238A1F40E94111A81FDD0C0E9
:102F300089E30E9490190E9441202FEF87EE93E0D1
:102F4000215080409040E1F700C0000089E315C0A7
:102F50008338C1F40E94111A80FDBAC083E50E9433
:102F600090190E9441202FEF81EE94E02150804083
:102F70009040E1F700C0000083E50E9462190E94C2
:102F80004120A6C08438A1F40E94111A82FDA0C07D
:102F900087E40E9490190E9441202FEF81EE94E077
:102FA000215080409040E1F700C0000087E4E5CF69
:102FB0008CEF8C0F813A40F580914802882319F0FC
:102FC000813051F01EC080918202823209F04CC0E3
:102FD0008C2F0E94951B46C0809182028232C1F3E1
:102FE000C43149F018F4CB3049F03AC0C93219F075
:102FF000C83321F035C01092480232C081E08170A0
:1030000031C01092480230C080E28C0F883068F4E2
:10301000C77081E090E001C0880FCA95EAF79091EF
:103020008202892B80938202AACFEBE5EC0FE3307A
:1030300040F4F0E0ED5CFE4F808190E00E94EC19DE
:1030400047C0C85ACB3108F043C0EC2FF0E0EE0F78
:10305000FF1FEA5CFE4F808191810E94C71938C032
:1030600080E0CDCF811134C0809102018130E1F444
:103070008091530287FF18C0EC2FE695E695E69500
:10308000F0E0E85DFD4F8281282F30E04C2F477043
:1030900081E090E002C0880F991F4A95E2F78223F1
:1030A0009323892B61F410C0E2E2F2E088E292E01F
:1030B0002191C21721F08E179F07D1F705C08C2FE1
:1030C0000E9462190E9441208C2F0E94901957CFB4
:1030D000CF9108951F93CF93DF93182FEB010E9498
:1030E0008D17209741F08FE99FE00197F1F700C01D
:1030F00000002197F6CF812F0E943C17DF91CF91DE
:103100001F9108958091010108950F931F93CF930C
:10311000DF938B01EA0190917B01943079F58F70F8
:103120008093E9008FEF9091E800815095FD06C0F3
:1031300095ED9A95F1F700008111F5CF8091E800A7
:1031400085FF1CC00E94C90F882361F08091E800B0
:103150008E778093E80012C0F80181918F018093EF
:10316000F1002197209791F38091E80085FDF4CF3D
:103170008091E8008E778093E800E4CFDF91CF91D3
:103180001F910F910895CF93DF93EC0148E050E039
:10319000BC0181E00E94851888E0FE01A1E7B1E052
:1031A00001900D928A95E1F7DF91CF91089581E02A
:1031B0008093E00080E28093D8001092C9008FE1F4
:1031C0009EE40197F1F700C0000087E090EBDC017E
:1031D0008093890290938A02A0938B02B0938C0211
:1031E0009CE088E10FB6F894A895809360000FBE2C
:1031F00090936000FFCF78941F920F920FB60F92BA
:1032000011248F939F93AF93BF9380915602909117
:103210005702A0915802B09159020196A11DB11D0B
:103220008093560290935702A0935802B09359028C
:10323000BF91AF919F918F910F900FBE0F901F90F4
:1032400018952FB7F89460915602709157028091AB
:103250005802909159022FBF08952FB7F89480918A
:10326000560290915702A0915802B09159022FBF77
:1032700008951F920F920FB60F9211248F939F9370
:10328000AF93BF9380915502811113C08091560274
:1032900090915702A0915802B09159024196A11DF8
:1032A000B11D8093560290935702A0935802B09399
:1032B0005902BF91AF919F918F910F900FBE0F90C8
:1032C0001F90189590910201913021F49091530232
:1032D00097FD03C0E0E2F2E01DC0E82FE695E69519
:1032E000E695EE31E0F4F0E0E85DFD4F877021E017
:1032F00030E0A90102C0440F551F8A95E2F7CA01C8
:1033000080959281892382830895319652E0E63236
:10331000F50729F092818913F8CF1282F6CF08952C
:10332000909102019130D1F49091530297FF16C011
:10333000E82FE695E695E695EE3140F5F0E0E85D9C
:10334000FD4F877021E030E0A90102C0440F551FF6
:103350008A95E2F7CA019281892B16C0A2E2B2E0F7
:10336000EFEF90E02D91821789F0EF3F19F42111D2
:1033700001C0E92F9F5F9630A9F7EF3F39F00E2E7D
:10338000000CFF0BE05EFD4F828308950895A3E0DB
:10339000B0E0EDECF9E10C94622120915102309102
:1033A000520228173907A1F09093520280935102DC
:1033B000E0914F02F0915002309751F024E02983C0
:1033C0009B838A830084F185E02DCE0101960995C7
:1033D0002396E2E00C947E21A3E0B0E0E2EFF9E175
:1033E0000C94622120914D0230914E02281739072A
:1033F000A1F090934E0280934D02E0914F02F09124
:103400005002309751F023E029839B838A83008404
:10341000F185E02DCE01019609952396E2E00C940A
:103420007E21E0914F02F0915002309729F00190F7
:10343000F081E02D0995089580E0089587E290E0FD
:103440000E94B1200895CF93C82F811102C06FEF61
:1034500001C065E284E290E00E94B120C11102C087
:103460006FEF01C061E085E290E00E94B120C111E0
:1034700002C06FEF01C064E186E290E00E94B120DB
:10348000CF91089584E290E00E949320853281F4E8
:1034900085E290E00E949320813051F486E290E032
:1034A0000E94932091E0843109F090E0892F01C0BF
:1034B00080E0817008950F931F93CF93DF93C42F03
:1034C000122FFC0185818823B1F040934C020E94A9
:1034D0002D1990934B0280934A0280E28C0F883022
:1034E00008F074C0C77081E001C0880FCA95EAF780
:1034F0000E9432176BC080914C02481349C0209142
:103500004A0230914B024FB7F89480915602909145
:103510005702A0915802B09159024FBF821B930BE2
:10352000883C9105A8F5D0E2D10FC117E9F080E2FF
:103530008C0F883040F4C77081E001C0880FCA95B5
:10354000EAF70E942B17D83080F581E0912F977011
:1035500001C0880F9A95EAF70E943217093359F58E
:1035600060E570E089E32AC0093319F460E570E092
:1035700002C060E070E0802F0E946A18D83030F5F9
:10358000212F277081E001C0880F2A95EAF70AC031
:1035900080E28C0F8830D0F4C77081E001C0880FC2
:1035A000CA95EAF70E942B1711C0093351F460E560
:1035B00070E089E309C060E070E0802F0E946A1823
:1035C000DFCF60E070E0802F0E946A18DF91CF911A
:1035D0001F910F910895CF93DF93C0E7D3E060E090
:1035E000CE010E94B1202196C11584E0D807B9F719
:1035F000DF91CF9108951F93CF93DF93962F84305F
:10360000E8F46730D8F44F30C8F4632F122FC42F7A
:10361000D0E0CC0FDD1F2EE1929FC00DD11D1124F3
:1036200092ED899FC00DD11D1124CE0188960E9474
:10363000B120612FCE0189960E94B120DF91CF91F8
:103640001F910895A0E0B0E0E8E2FBE10C945A215C
:10365000A12CE12CF12CB12C00E010E0C0E0D0E076
:103660006701C00ED11EFE01EE0FFF1FEC0DFD1D08
:10367000E651FC4F259134914C2F6B2D8A2D0E94E1
:10368000FB1A2196CF30D10571F7025E1F4FB3941C
:1036900087E0B812E3CF82EDE80EF11CA39484E03A
:1036A000A812D9CFCDB7DEB7EAE00C94762180E03E
:1036B0000E94231A60E070E0CB010E941E1A0E9453
:1036C000221B0E94EB1A81E00E94231A08950F9397
:1036D0001F93CF93DF93843008F56730F8F44F30B1
:1036E000E8F4C42FD0E0CC0FDD1F2EE1629FC00DA7
:1036F000D11D112432ED839FC00DD11D1124CE01A7
:1037000088960E94932090E0182F0027CE0189967A
:103710000E9493209801282BC90102C080E090E00C
:10372000DF91CF911F910F910895482F50E0FA013A
:103730003597EF33F10508F072C0E855FF4F0C9450
:103740002B210E94CD1F65C080914902817F8E7F11
:103750008093490281E08093480208950E940917EE
:103760002FEF84E39CE0215080409040E1F700C0BF
:1037700000000E94D71880914902982F909591706F
:1037800090FB80F980934902911143C0897F877F24
:1037900010C08091490281FB222720F991E09227F5
:1037A00090FB81F980934902992399F18091490214
:1037B0008160809349022DC08091490282FB2227BB
:1037C00020F991E0922790FB82F9ECCF8091490299
:1037D00083FB222720F991E0922790FB83F9E2CF27
:1037E0000E9409178091530287FB222720F991E05C
:1037F000922790FB87F9809353020BC0895391E085
:1038000001C0990F8A95EAF7892F0E9406170E9436
:10381000091781E008958D51F2CF81E0F6CF80E065
:103820000895A0E0B0E0E7E1FCE10C945821843079
:1038300030F4811105C0909190009F7704C083E01F
:1038400090919000906890939000A0919600B09114
:103850009700282F30E00E94382123E030E040E03C
:1038600050E00E9409210027122F232F342F012F0F
:10387000122F232F332780919600909197006CE0B0
:1038800070E00E94F5206017710730F0C80169E010
:1038900070E00E94F5205EC08091960090919700A4
:1038A000E0909600F0909700E0919600F0919700DC
:1038B000C6E0D0E0BE010E94F520060F171F211DB3
:1038C000311D4801590185E0880C991CAA1CBB1CBC
:1038D0008A95D1F7C701BE010E94F5206F01E12C46
:1038E000F12CA7019601260F371F411D511DC5015F
:1038F000B4010E94092169017A01E0919600F091DA
:103900009700CA01B9010E94E5209B01AC01DF01CB
:103910000E9447219B01AC01C701B6010E94E5202E
:10392000DC01CB012FE0B695A795979587952A9551
:10393000D1F7009196001091970020E030E0081731
:1039400019072A073B0728F46091960070919700A9
:10395000CB01BC017093990060939800CDB7DEB79E
:10396000ECE00C947421682F86E090E00E94B12076
:10397000089580E008959091530292FF10C041E0B5
:10398000282F2471243009F040E031E0282F2871DD
:10399000283009F030E0431711F02CE0822793FF24
:1039A00010C041E0282F2471243109F040E031E0BB
:1039B000282F2871283109F030E0431711F02CE04E
:1039C00082273091540230FF10C051E0282F21711E
:1039D000213009F050E041E0282F2871283009F00B
:1039E00040E0541711F029E0822731FF10C041E078
:1039F000282F2171213109F040E031E0282F287172
:103A0000283109F030E0431711F029E0822794FDB6
:103A1000877E08958238910569F1B0F4813391056C
:103A200009F475C048F48932910509F467C08A32F7
:103A3000910509F471C008958533910509F459C0C1
:103A400089339105B9F00895833E910589F138F4E1
:103A5000803E9105D1F0823E910529F10895863E80
:103A60009105C9F1873E9105D9F1843E910509F090
:103A70006CC027C02091530220FD57C021FD55C0C6
:103A80002091540223FD5BC008958091530280FD74
:103A900048C08091540280FF48C08091530284FD49
:103AA00046C083EE51C08091530282FF3CC0F5CFE7
:103AB0008091530282FD37C08091540280FD35C051
:103AC000ECCF8091540281FF36C08091530284FD77
:103AD0002EC087EE39C08091530283FF2AC0F5CFF4
:103AE0008091530283FD25C08091540281FD23C043
:103AF000ECCF8091530285FD22C01FC080915302FC
:103B000085FD1BC08091540283FF19C00AC08091BB
:103B1000530286FD16C017C08091530286FD13C064
:103B200010C089E311C082EE0FC080EE0DC080E0AE
:103B30000BC086EE09C084EE07C085E305C089E2AC
:103B400003C08AE201C081E390E00895F894E82F71
:103B5000E295EF70F0E031A1282F2F7081E090E026
:103B600001C0880F2A95EAF7982F9095932391A387
:103B700092A1892B82A378940895AEE0B0E0E3ECA3
:103B8000FDE10C945421AE014F5F5F4F7A018EE04E
:103B9000FA0111928A95E9F70DE111E06A0194E2C8
:103BA000492E91E0592E66246394712C33E3832EC1
:103BB00031E0932EF80180818F3F09F446C0F894DC
:103BC000E82FE295EF70F0E021A18F70A30102C011
:103BD000440F551F8A95E2F7CA01922F982B91A3A3
:103BE00092A18095892382A3789400C0E4E2F1E059
:103BF00021E030E0A12CB12C41914F3F89F0A42F5E
:103C0000A295AF70B0E090968C9190E04F7002C09A
:103C1000959587954A95E2F780FD02C0C90102C0DB
:103C200080E090E0A82AB92A220F331F8E169F0643
:103C300019F7F80180818F3F11F00E94A61DF0EA6C
:103C4000FA95F1F7F601B182A0820F5F1F4FF2E003
:103C5000CF0ED11C4016510609F0ACCF4EE050E01B
:103C6000B70185E891E00E948921892B91F08EE0CF
:103C7000F701A5E8B1E001900D928A95E1F781E0A6
:103C8000809388020E942D19909387028093860268
:103C900017C080918802882399F020918602309184
:103CA00087024FB7F8948091560290915702A091E5
:103CB0005802B09159024FBF821B930B059710F425
:103CC00080E018C04EE050E065E871E083EA91E0E2
:103CD0000E948921892B59F08EE0E5E8F1E0A3EA02
:103CE000B1E001900D928A95E1F781E001C080E09A
:103CF000109288022E96E0E10C947021773048F4FF
:103D00006F3038F4843028F4462F672F0E94671BE9
:103D1000089580E090E008951F93CF93DF930E9471
:103D20000A1DEC01C11580E5D807E8F5C11590E43E
:103D3000D90708F0A8C0C03ED10530F5CD3CD1056B
:103D400008F094C0C83AD10578F4C53AD10508F016
:103D500083C0C130D10509F47CC008F4F2C0C4307E
:103D6000D10508F0F1C0EDC0C33CD10508F0E9C0B1
:103D7000C85AD0E0CC0FDD1FCA5CDE4F0990D88155
:103D8000C02DCE019464E1C0C11580E2D80708F0CF
:103D9000CBC0C11591E0D90708F06BC0C83ED10572
:103DA00008F4D2C0CEC0C03682E5D80728F5C034AA
:103DB00092E5D90708F079C0C03282E5D80708F04B
:103DC0006CC0C11592E5D90708F481C04C2F469507
:103DD000469580E2489FA0011124C37021E030E0A5
:103DE000C90102C0880F991FCA95E2F7EA01C82BE2
:103DF000D92BCE019D68A9C0C03A82E5D807B8F496
:103E00008C2F8F71C03892E5D90708F07BC086955A
:103E1000869590E2899F90011124C37081E090E023
:103E200002C0880F991FCA95E2F79A6868C0C03C23
:103E300082E5D80708F46DC0C03E92E5D90708F0C6
:103E400080C0CF71DD27DC2FCC27CE01806F906A38
:103E50007CC081E090E079C0C55AD0E0CD5CDE4FF7
:103E60008881C82FD0E0CE0190646FC0CE019065EC
:103E70006CC08D2F0E94BB1C182FCE0199270E9469
